:020000040000FA
:020000002528B1
:080008008C00030E83018D0042
:100010000A088E008A0104088F000E281408810047
:100020000130160296009608031D1B28150896003D
:100030000130170297000B110F0884000E088A0088
:100040000D0E83008C0E0C0E0900FF309100FF3066
:1000500092009211FD201212FC209212FB209311AB
:10006000F7201312F6209316F520DF300121F3203C
:10007000892098008920990089209A005A309B0095
:10008000051A49280230B420F3209312861E9316D5
:10009000F5209B0B402818089B009B0803195B2840
:1000A00000309C0000309D0078209D0B54289C0B54
:1000B00052289B034D2819089B009B0803196728A9
:1000C00000309C0078209C0B62289B035D281A0856
:1000D0009B009B0803196F2878209B03692813163F
:1000E000F620F3200130BB201312F6202F287728AA
:1000F000861C82280130C220861C8228D83001212B
:1001000081288028F3200130B4209312861E931694
:10011000F52808309C0003109B0D97201B049B00C2
:10012000F3209312F5209C0B8B281B08080006195E
:100130009E28061D99280130DB2097280130DB20FE
:100140009D01861CA52801309D009315F720061DF2
:10015000AE280619A9280130DB20A7280130DB20B2
:100160009311F7201D0808009E001E089F006430B0
:10017000A0006430C9289B001B089F006430A000C9
:100180003230C9289E001E089F006430A000013054
:10019000C928A100FF30A2002008A4001F08A30066
:1001A000173022070318D128A30BD028A40BCE2880
:1001B000A10BCC2808009E001E089F009F08031971
:1001C000E5283230E6209F03DE280800A000F43046
:1001D000A100FC30A20020082107031C00342207E4
:1001E0000318EF28080064000800F828F828F82809
:1001F000130886000800FE28FE28FE281208660064
:0A02000008009E001E0862000800BE
:02400E00F53F7C
:00000001FF
